:10000000CBC20000E6C20000E4C20000E2C2000071
:10001000E0C20000DEC20000DCC20000DAC2000064
:10002000D8C20000D6C200000C9494200C94602129
:100030000C94731ACEC20000CCC20000CAC20000E9
:10004000C8C20000C6C20000C4C20000C2C2000094
:10005000C0C200000C94EA1ABCC20000BAC2000080
:10006000B8C20000B6C20000B4C20000B2C20000B4
:10007000B0C20000AEC20000ACC20000AAC20000C4
:10008000A8C20000A6C20000A4C20000A2C20000D4
:10009000A0C200009EC200009CC200009AC20000E4
:1000A00098C2000096C2000094C2000029002B00F4
:1000B000E000E100510000001E003600040037009F
:1000C00052004D001F0034001200140000042A00EA
:1000D0002000330008000D00E1042C002100130073
:1000E00018000E00E3004A0022001C000C001B0058
:1000F00000000000645263520000000F0000557CB5
:10010000000061520000000700004C0023000900BD
:10011000070005000000490024000A000B00100041
:10012000E6004B002500060017001A00E4002152EB
:10013000260015001100190000002C0027000F00F8
:1001400016001D0050004E002A0028003800E5006F
:100150004F000000000000000100225200000000DB
:100160003A002F004D7E4E7E000000003B00587E7E
:10017000457E517E010000003C00547E467E487E54
:10018000010001003D00577E477E1E020100000075
:100190003E00537E437E597E0000000000000000B8
:1001A000000000000000000000000100000000004E
:1001B000000000003F00607E497E22020000000037
:1001C00040006400557E5E7E0100000041004C7ED0
:1001D000567E5F7E010000004200447E427E507EDB
:1001E0000000010043002D0032000000000000006C
:1001F000440045004F7E01000000000000000000A8
:10020000000000000000000000002F0200000000BD
:1002100000000000000000000000000000000000DE
:10022000000000005B7E00000000010000000000F4
:10023000527E0000000000000000000000000000EE
:1002400000000000000000000000000000000000AE
:10025000000000000000000000000000000000009E
:100260000000000000000000000030004A7E5A7EBE
:1002700000000000000000002E004B7E0000000087
:10028000000000005C7E0000000001000000000093
:100290005D7E000000000000000000000000000083
:1002A0000000000001000100010001000100000049
:1002B000000000000000000001000100000000003C
:1002C000CF000000010001000000CD00CE000000C2
:1002D0000100010000000000D0000000010001004A
:1002E00000000000000000000000537C000001003E
:1002F000000000000000547C00000000000000002E
:100300000000567C00000000370036000000577CDB
:100310000000240021001E0027000100000025002D
:1003200022001F000100D200000026002300200050
:100330000000D10000002D000000000001000100BD
:1003400001000100010001000100000001000100A6
:1003500001000100010000001E00140004001D0047
:10036000010001001F001A0016001B00010001001F
:100370002000080007000600010001002100150010
:100380000900190001000100220017000A00050001
:100390000000010001000100000001000000010058
:1003A00000000000000001000000010023001C000C
:1003B0000B00110000000100240018000D001000C7
:1003C0000100010025000C000E00360001000000B5
:1003D000260012000F003700010001002700130063
:1003E0003300380001000100010001003400010069
:1003F0000100000016034500720067006F00440012
:100400006F007800200045005A00000028035A00C1
:1004100053004100200054006500630068006E0036
:100420006F006C006F006700790020004C006100D5
:100430006200730000000403090409025400030170
:1004400000A0FA09040000010301010009211101C3
:10045000000122440007058103080001090401008E
:1004600001030102000921110100012247000705D3
:1004700082031000010904020001030000000921A9
:1004800011010001226D0007058303200001120104
:1004900000020000000897327449010001020001C7
:1004A00005010980A101850319012AB7001501265C
:1004B000B700950175108100C0050C0901A10185E7
:1004C0000419012AA002150126A0029501751081C8
:1004D00000C005010906A1018506050719E029E705
:1004E000150025019508750181020507190029EFFE
:1004F0001500250195F075018102050819012905EE
:10050000950575019102950175039101C0050109D9
:1005100002A1010901A100050919012908150025F9
:100520000195087501810205010930093115812500
:100530007F95027508810609381581257F9501751B
:10054000088106050C0A38021581257F950175087A
:100550008106C0C005010906A101050719E029E7C8
:100560001500250195087501810295017508810125
:100570000507190029FF150026FF0095067508815B
:10058000000508190129051500250195057501913A
:1005900002950175039101C011241FBECFEFDAE06F
:1005A000DEBFCDBF11E0A0E0B1E0E0E4F8E402C0BE
:1005B00005900D92A639B107D9F722E0A6E9B1E07E
:1005C00001C01D92A33FB207E1F70E9408140C94EA
:1005D000A62316CD8098889A8198899A84988C9AB7
:1005E00085988D9A86988E9A87988F9A08952098E4
:1005F00028982198299822982A9823982B985298DD
:100600005A9853985B983E984698089544D18093A1
:10061000000110920101EBDFDDCFA1E0B0E0E3E1EA
:10062000F3E00C942A238091000190910101892B21
:1006300081F0809198018F5F80939801811109C0AA
:100640002AD190E08093000110920101892B09F4D6
:10065000C4D086ECE82E82E0F82EC12CD12CA12C3F
:100660008C2D895FB82E8091000190910101892B1A
:10067000B9F481E00C2C01C0880F0A94EAF7809548
:10068000898304E610E021E030E0CE010196AC0160
:1006900062E180E40E947B1C809300019093010141
:1006A0008B2D8B3009F45CC008F04CC0893009F404
:1006B00051C08A3009F451C0883009F448C0209AEA
:1006C00028988091000190910101892B09F04EC07A
:1006D000198224E630E041E050E0CE010196BC01F1
:1006E00080E40E94091C809300019093010189819C
:1006F00080958F73F7019081891719F08083AA2460
:10070000A3949FB18FB1869586958C739370892B36
:100710009FE38927F7019781891719F08783AA2416
:10072000A39465DF8FEFC81AD80A8FEFE81AF80A8A
:1007300087E0C816D10409F093CF8A2D2196EAE00C
:100740000C9446238C3079F4539A5B98BACF219A53
:100750002998B7CF229A2A98B4CF239A2B98B1CF51
:10076000529A5A98AECF3E9A4698ABCF80E0C1CF0E
:1007700092D0809300011092010139DF2BDFE4ED6C
:10078000F2E08EE011928A95E9F70895259A2D9A64
:100790000895269A2E9A0895279A2F9A0895569882
:1007A0005E98089525982D98089526982E98089576
:1007B00027982F980895F3DFF5DFF7DFF9CF90E062
:1007C000909389008093880090938B0080938A0097
:1007D00090938D0080938C000895EDDF8FEFEFDF15
:1007E000D5DF8FEF90E722E0815090402040E1F785
:1007F00000C00000CEDF8FEF90E722E081509040F4
:100800002040E1F700C00000C7DF8FEF90E722E053
:10081000815090402040E1F700C00000C3DF8FEF1F
:1008200090E722E0815090402040E1F700C00000B6
:10083000BCDF8FEF90E722E0815090402040E1F74D
:1008400000C00000B5DFB7CF89EA8093800089E05F
:100850008093810024982C983F98479A54985C9AEA
:1008600055985D9A6E98769A0E94E50F6093B20251
:100870007093B3028093B4029093B50267702FEF28
:10088000629FC0011124959587959595879597DF6F
:10089000A4DF0C945B13A2E0B0E0E1E5F4E00C947B
:1008A000302380E280930001109201018091990130
:1008B00081110EC00E94961B81E0809399018FEFF9
:1008C00093ED20E3815090402040E1F700C000000C
:1008D0009FE319829A8304E610E022E030E0CE0123
:1008E0000196AC0160E080E40E947B1C9C01809337
:1008F000000130930101892B71F422E030E0CE0138
:100900000196AC016CE080E40E947B1C9C0180930A
:10091000000130930101822F2296E4E00C944C23D5
:100920001092B2021092B3021092B4021092B50269
:1009300084E080618093B20264E170E080E090E046
:100940000E94E70F0C94B20F0C945C13089582542C
:100950009E47FC014F9760F4E855FC4DDB0115966E
:100960008C910C941C23811519F08FE192E05AD1DF
:1009700081E008958115E1F380E292E0F8CF8115DE
:10098000B9F383E292E0F3CF811591F384E292E030
:10099000EECF811569F385E292E0E9CF811541F34D
:1009A00086E292E0E4CF811519F387E292E0DFCF8F
:1009B0008115F1F28DE292E0DACF8115C9F28EE273
:1009C00092E0D5CF8115A1F280E392E0D0CF8115DE
:1009D00079F284E692E0CBCF811551F286E392E082
:1009E000C6CF811529F287E392E0C1CF811509F4C2
:1009F000BFCF88E392E0BBCF811509F4B9CF81E383
:100A000092E0B5CF811509F4B3CF8FE194E1AFCF78
:100A1000811509F4ADCF80E294E1A9CF811509F4E5
:100A2000A7CF81E294E1A3CF811509F4A1CF84E29D
:100A300094E19DCF811509F49BCF85E294E197CF96
:100A4000811509F495CF86E294E191CF811509F4DF
:100A50008FCF87E294E18BCF811509F489CF84E6AB
:100A600094E185CF811509F483CF8DE294E17FCFA6
:100A7000811509F47DCF80E394E179CF811509F4E4
:100A800077CF88E094E173CF811509F471CF8FE1BE
:100A900096E16DCF811509F46BCF86E194E167CFC4
:100AA000811509F465CF86EE2CD280E317D386EE4C
:100AB000ADD28CE213D35CCF811509F459CF81EE0E
:100AC00020D280E30BD381EEF3CF811509F450CF10
:100AD00081EE17D28EE2F6CF0895CF93DF93EC012B
:100AE0005EDE60DE62DE64DECE017CD18150873066
:100AF00038F4E82FF0E0E953FC4D0C941C2346DE5B
:100B0000CE01DF91CF91089541DE43DEF9CF3EDE85
:100B100043DEF6CF3BDE3DDEFBCF8530C8F46E30E2
:100B2000B8F44630A8F450E096E0699F400D511D9E
:100B3000112494E5899F400D511D1124FA01EE0FF7
:100B4000FF1FE455FF4F85919591282F822F08951F
:100B500021E090E0FBCFE1CF08959C0191509F31BF
:100B6000B0F4832F817034FF0AC08295807F31FDFD
:100B7000806232FD806433FF0BC08068089531FDD0
:100B8000826032FD846033FF03C08860089580E096
:100B90000895CF93DF93EB01E0DFFE010995DF912C
:100BA000CF910895CF93DF93EC01805E9109089770
:100BB00020F064E77AE0209711F465E778E0CE0151
:100BC000E8DF8C2F9ED1DF91CF910895CF93DF93F3
:100BD000EC011CD2CE01805E9109089720F069E7F4
:100BE0007AE0209711F46AE778E0CE01D2DFDF9156
:100BF000CF9108950F931F93CF93DF938C01EB0157
:100C0000D1DF209739F4C801E1DFDF91CF911F9147
:100C10000F9108958FE99FE00197F1F700C0000060
:100C20002197EFCF60E570E08933910511F060E026
:100C300070E0E0CF81E0089581E00895FBCF089552
:100C400081E0089584CE089508950895FDCF089514
:100C500008950895A6E0B0E0E0E3F6E00C943123B7
:100C600049835A839E8330919F0189819A813111F2
:100C700017C03E81311589F0211579F085D5182FDF
:100C8000682F89819A815FD569817A81812F0E943D
:100C9000B6112696E3E00C944D2366D5182FF4CFB9
:100CA00073D569817A81F3CFFC01262F4081518170
:100CB0006281738184819581CDCFCF93DF93EC01E5
:100CC00061E0F2DFBE01B8DF811529F061E0CE01FD
:100CD000EBDFBE01B3DFDF91CF9108950F931F9338
:100CE000CF93DF93EC0160E0DFDF8C01BE01ADDF6D
:100CF000BE01C801ABDFDF91CF911F910F91089525
:100D00000F931F93CF93DF93EC0161E0CDDF8C0154
:100D1000BE0196DF811106C080E0DF91CF911F9167
:100D20000F910895BE01C8018DDF8115A9F3BE01A1
:100D3000C8010E94CA17811579F3BE01C8010E943B
:100D40004414811549F3BE01C8010E941D14811588
:100D500019F3BE01C8010E94B9128115E9F2BE0162
:100D6000C8010E94CB128115B9F2BE01C8010E94D0
:100D7000E512D3CF21E030E002C0220F331F8A9565
:100D8000E2F7C9011DC4CF93C82F81E090E00C2E7B
:100D900002C0880F991F0A94E2F70E94DF0F8C2F80
:100DA000E9DFCF91089581E0089581E00895FBCFB8
:100DB0000895CF93C82FB3D38C2FF7DF8C2FF7DF95
:100DC000CF91089581E0F5DF0C940E1B80E0F1DFF8
:100DD0000C943F1B3DDF0E941B1A36C037D039DF11
:100DE0000C941E1A292F30E048E0911102C09C019A
:100DF00040E0C90164E0969587956A95E1F7009710
:100E000011F04C5F9C01C901969587959695879541
:100E1000009711F04E5F9C01C90196958795840F4C
:100E2000089581E008950895CF93DF93C82FF9DFE7
:100E3000D82F811511F08C2FF6DF8D2FDF91CF91F8
:100E400008950895F1CF089580E0FCCF0E9418180E
:100E5000F9CFCF930E941818C82F80919A018C1750
:100E600071F0C0939A010E94DE1A60939B01709307
:100E70009C0180939D0190939E018C2FE3DFCF9185
:100E80000895ADE0B0E0E7E4F7E00C943223488742
:100E900059876A877B878C879D87911183D71F82AB
:100EA00086E0FE0138969E012F5F3F4FD9010190E9
:100EB0000D928A95E1F78D8181110CC029813A81CB
:100EC0004B815C816D817E818F81B7D62D96E2E06A
:100ED0000C944E23CE010196F0DE8111EFCFF6CFB8
:100EE000FC012481213019F48081918180C408950E
:100EF000611521F00E949D150C9452160E94DD157B
:100F0000FBCFCF93C82F8115B9F08238B9F40E9476
:100F1000271881FD11C089E30E944F19CED78FEFAA
:100F200097EE23E0815090402040E1F700C00000A0
:100F300089E30E946619C1D7CF910895833899F447
:100F40000E94271880FDF8CF83E50E944F19B5D77E
:100F50008FEF91EE24E0815090402040E1F700C0F7
:100F6000000083E5E6CF843899F40E94271882FDBB
:100F7000E3CF87E40E944F19A0D78FEF91EE24E0D2
:100F8000815090402040E1F700C0000087E4D1CFBD
:100F90008450813A68F48C2F0E94C918811521F081
:100FA0008C2F0E94661989D78C2F0E944F19C3CFAE
:100FB0008C2F805E883048F481E0C1FD84E0C0FD64
:100FC000880FC2FD8295CFD6B6CF8C2F855A83303D
:100FD00030F48C2F8452990B0E945518ADCFEC2F12
:100FE000E85AEB3150F4F0E0EE0FFF1FE55EFE4FE4
:100FF000808191810E947C189FCF8C2F8D5C8331E2
:1010000008F09ACF61E08C2F73DF96CF811509F439
:101010004EC0823861F40E94271881FF48C089E3DE
:101020000E944F194AD789E30E94661946C7833840
:1010300051F40E94271880FF3AC083E50E944F199F
:101040003CD783E5F1CF843851F40E94271882FF02
:101050002EC087E40E944F1930D787E4E5CF982F40
:101060009450913A08F3982F905E983050F4982F4E
:1010700081E091FD84E090FD880F92FD829579D604
:10108000D5CF982F955A933020F480E090E00C94BF
:101090005518982F985A9B3120F480E090E00C94DA
:1010A0007C18982F9D5C933110F460E021CF089557
:1010B0001F93CF93DF93182FEB0123DF209731F499
:1010C000812FA4DFDF91CF911F9108958FE99FE0D9
:1010D0000197F1F700C000002197F0CF60E570E0C4
:1010E000893311F060E070E0E3CF811511F03BD659
:1010F000E4C60895811511F03CD6DFC60895A0E03E
:10110000B0E0E5E8F8E00C942C236C01D62FC72F53
:10111000FC011581068102950F701AD6E82E811503
:10112000E9F0E12E1115D1F08C2F807F803461F031
:101130008D2F805E8830E0F08C2F807E803221F40D
:10114000D230B0F00115A1F08091C50282FF10C02D
:1011500082E0D7D6FDD591E08927E82EEC2FE295E5
:10116000EF70C03C78F5F0E0E253FC4D0C941C238A
:10117000E12CF4CF0C2F0F70C03110F00295007FDE
:10118000111581F0011549F08D2F805E883010F027
:10119000D11105C0802FE7D590D68D2F40C0802F6C
:1011A000F3D5FACF8D2F32DF011561F08D2F805EE0
:1011B000883010F0D11103C0802FDBD502C0802F02
:1011C000E9D57BD6E11409F4B2C0BED580FDAFC02D
:1011D000F6011582B3D522D2C60168D1AFD52CD283
:1011E000A6C08C2F8F70F82EC07FC03219F0F294F9
:1011F00080EFF822D13038F079F1111509F437C0B9
:101200000115C9F0CACF8091C50282FD10C0111529
:1012100041F0F11419F08F2DA6D54FD680E071DE84
:10122000D1CF80E0F3DEF11469F28F2DC6CF111516
:1012300051F0013018F48F2D58DFC4CF09F0C2CF20
:101240008F2DC4D5BFCF0111BDCF8F2D53DF8F2D73
:10125000C8D58F2DADD5B6CF111521F0023008F0CD
:10126000B1CFE9CF0111AECF8F2D44DFABCF011548
:10127000D9F3D93349F48FEF97EE23E081509040B2
:101280002040E1F700C000008D2FC0DE9BCF8C2FE7
:10129000869586958370813060F009F093CF8D2F0D
:1012A0009C2F9370111102C080E090E00E947C1886
:1012B00089CF8D2F9C2F9370111102C080E090E098
:1012C0000E9455187FCF612F8D2F12DE7BCF8C2F80
:1012D0008370C1F5111128C04D2F42954695477076
:1012E000440F440F2D2F2F7030E0042E02C0220F28
:1012F000331F0A94E2F780E090E0D4FF09C08FE04A
:1013000090E002C0880F991F4A95E2F7809590956A
:10131000C695C695C370822B932BC23079F0C3302B
:1013200079F0C13049F055D10E9418188BDDCDB746
:10133000DEB7E8E00C94482345D1F6CF51D1F4CF85
:101340003FD1F2CF111559F1C0FFEECF4D2F42958D
:1013500046954770440F440F2D2F2F7030E0042E18
:1013600002C0220F331F0A94E2F780E090E0D4FF1E
:1013700009C08FE090E002C0880F991F4A95E2F7FC
:1013800080959095C695C695C370822B932BC230DD
:1013900061F0C33061F0C13031F073D1C5CF82301C
:1013A00008F4C2CFD3CF66D1BFCF72D1BDCF23D186
:1013B000BBCFCF70111529F08C2F30D18D2F95DE3A
:1013C000B3CF8D2F97DE8C2F37D1AECFD23F39F1EF
:1013D00068F4D03FC1F0D13F89F0111509F43FC046
:1013E000011509F439C08D2F8CDD9ECFD33FE9F074
:1013F000D43F99F78091C50282FD1FC08C2F8F7159
:10140000111511F310C0111531F001118DCF8C2F72
:101410008F7122D189CF023008F086CFF8CF8C2F80
:101420008F711111D1CFFAD07FCF111521F08C2FF0
:101430008F71EBD079CFE6D077CF111529F063E02B
:101440008C2F8F7147D570CF81E05BD5023008F4C7
:101450006BCF82E056D568CF8C2F8F71E4CF01150A
:1014600071F0D93349F48FEF97EE23E0815090402B
:101470002040E1F700C000008D2FC8DD55CF8C2F34
:101480008F71A2CF0F931F93CF93DF93EC016881ED
:1014900079818D81B5D18C0102D191D0B801CE0175
:1014A0002EDEDF91CF911F910F910895CF93DF939F
:1014B000EC018C81811581F0CE0122DC81110FC0FD
:1014C00047D4811549F08D81811531F08091C50295
:1014D00082FF02C082E015D5DF91CF910895CE0141
:1014E000D1DFCE01FBDBF8CF811511F04DD4E5C47F
:1014F0000895811511F04ED4E0C4089580E090E085
:101500000E94551880E090E00E947C184BD4D5D4FE
:101510000E946B160C9452160E947D19EFCF31D4A5
:10152000FBCF282F92959F70963099F060F4925FD0
:101530009F70923030F4203FB1F038F481E0283EC3
:1015400038F080E008959A5FF3CF81E0243FC9F737
:10155000089591E0813F09F090E081E0283E08F095
:1015600080E0892B089581E00895FC0124812115F4
:1015700021F0808191813BD1D4CF80E00895A6E015
:10158000B0E0E5ECFAE00C9432232696E2E00C940D
:101590004E23A7E0B0E0EFECFAE00C94322327965C
:1015A000E2E00C944E230895FECF0895FDCF0895F8
:1015B000FADFFCDF8093CE019093CF010895089568
:1015C000F7CF08952091CE013091CF01822B932B3C
:1015D000EFCF2091CE013091CF0182239323E8CF2A
:1015E0002091CE013091CF0182279327E1CF75CA98
:1015F0000895D9CF0895FDDFFADF8093CC01909351
:10160000CD01089580E090E0F6CF21E030E002C007
:10161000220F331F8A95E2F7C901EDCF21E030E0B8
:1016200002C0220F331F8A95E2F78091CC0190917E
:10163000CD01822B932BDFCF21E030E002C0220FBF
:10164000331F8A95E2F7209530958091CC019091D7
:10165000CD0182239323CFCF21E030E002C0220FBF
:10166000331F8A95E2F78091CC019091CD018227BA
:101670009327C1CF2091CC013091CD01822B932BA8
:10168000BACF2091CC013091CD0182239323B3CFE7
:101690002091CC013091CD0182279327ACCF0895C2
:1016A000CF93C1E061FDC4E060FDCC0F62FDC29547
:1016B00093E0769567959A95E1F7660F771F660F29
:1016C000771F460F571FFA0140E050E090E061910C
:1016D000DF019C01042E02C0369527950A94E2F79B
:1016E0002695220B26272C2326272E934F5F5F4F0C
:1016F0004430510561F7CF910895A82FA77023E0DA
:10170000969587952A95E1F7880F991F880F991F5D
:10171000680F791FFB0140E050E080E0219130E04C
:101720000A2E02C0369527950A94E2F72170042EFE
:1017300001C0220F0A94EAF7822B4F5F5F4F4430BB
:10174000510561F70895262F9E3068F4863058F4CD
:10175000682F70E086E0989F600D711D112440EAAB
:1017600051E0822F9DCF0895292F9E3058F4863066
:1017700048F490E060EA71E036E0239F800D911D0F
:101780001124BBCF80E00895CF92DF92FF920F9398
:101790001F93CF93DF936C010091CC011091CD0189
:1017A0008091CE019091CF01082B192BCFE0D0E092
:1017B00081E090E00C2E02C0880F991F0A94E2F796
:1017C00080239123892B61F4219790F7F12C8F2DA1
:1017D000DF91CF911F910F91FF90DF90CF900895EF
:1017E000FC2EB6018C2FCDD5019771F3F0CFCF939E
:1017F000DF93EC01C9DFBE01C4D5DF91CF9108951D
:101800000F931F93CF938B0190919F01911531F00E
:10181000CB01EDDFCF911F910F910895811551F00C
:10182000CB01B2DFC82F682FC8018DDFB8018C2F24
:10183000A8D5F0CFCB0198DFC82FF8CF0F931F9317
:101840000091D0018091D101801303C01F910F91AD
:10185000089587E0089FF0011124EE52FE4F208189
:1018600031814281538164817581868192DE0F5F6F
:101870001F4F0770E7CF20910A0230910B02409171
:101880000C0250910D0260910E0270910F02809136
:1018900010027FCE80911002803170F480910F028F
:1018A000811551F0E091D0012091D10130910B02CE
:1018B00040910A022E1301C00895BF0187E0E89FFE
:1018C000F0011124DF01AE52BE4F14968C91149793
:1018D000811549F111968C911197831324C08C9135
:1018E000841321C015968C91159781111CC01296F6
:1018F0008D919D91A0910C02B0910D028A1B9B0BC2
:10190000883C910580F4809110028F7080618093F3
:101910001002E852FE4F80818F70806180838AE0E0
:1019200092E0C4DD8BCF6F5F7F4FFB01E770C2CFCA
:10193000E091D0019091D101E91302C080E00895B7
:101940009F0157E0E59FF0011124EE52FE4F5181B7
:10195000561306C05081581303C05581541305C057
:101960002F5F3F4FF901E770E7CF81E008958F9235
:101970009F92AF92BF92DF92EF92FF920F931F93CD
:10198000CF93DF93CDB7DEB72D970FB6F894DEBFB8
:101990000FBECDBF8C0186E0F801DE0118960190E4
:1019A0000D928A95E1F7F801F58084819AE0892EFD
:1019B00092E0992E90910E02911117C0811509F4B1
:1019C000EFC0F11409F42EC1C801CFDD811509F46F
:1019D00029C187E0F801D40101900D928A95E1F7C1
:1019E000C4017EDA57DF47DFDBC0E080A280B3802E
:1019F000D0900F0220910C0230910D02A501421BE4
:101A0000530BD11409F4CFC0483C510508F09EC0D7
:101A1000811509F4C5C090910B029180809110024C
:101A2000803108F065C0991226C090910A029E117B
:101A300022C0F11057C08F708061809310021BDFAD
:101A40008AE092E033DD80911002F8018683F12C68
:101A50008F2D2D960FB6F894DEBF0FBECDBFDF9150
:101A6000CF911F910F91FF90EF90DF90BF90AF90BB
:101A70009F908F900895F11035C040E0692D8E2D14
:101A800057DF40E0692D8E2D53DFF82E8111DFCF17
:101A900088859985ACDE292F22952F70903450F4DB
:101AA0009F70223078F0911591F0F8019681903175
:101AB00070F4CECF2A5F2F70223070F0C801F6DCB0
:101AC000FD2CC6CF911519F0811509F4C1CF805EA8
:101AD000883008F4BDCFF2CF803F08F4B9CF815FE2
:101AE0008330F7CF80911002816080931002AFCFD6
:101AF000991207C090910A029E1103C0F11409F4D3
:101B000073C0C80132DD811509F48CC0F11409F4E9
:101B100089C080911002803280F020910A023091B9
:101B20000B0229833A83AB82BC8290910E029D8383
:101B30001E828F83CE010196B9DC87E0F801AAE00E
:101B4000B2E001900D928A95E1F74CCF909110028E
:101B5000903188F4488559856A857B858C859D857B
:101B60000EDD8AE092E0A2DCF40187E011928A9512
:101B7000E9F781DE6CCF811599F020910B0281810C
:101B80002813BFCF80910A028E11BBCFF110B9CFBD
:101B90009683C8018BDCF40187E011928A95E9F7FE
:101BA000FF24F39455CF483C510508F03EC0811501
:101BB000B9F3F114B9F190910B028181981329C006
:101BC00080910A028E1125C08091100280FD18C0FC
:101BD0008031B0F08683807F803F39F08681982FF6
:101BE000907F905F8F70892B8683C8015FDC87E0D0
:101BF000F801AAE0B2E001900D928A95E1F7F3CEE8
:101C000087E0F801AAE0B2E001900D928A95E1F731
:101C1000C7CFC801AADC811190CF809110028160EA
:101C200080931002C80142DCBBCF488559856A8584
:101C30007B858C859D85A3DC97CFAEE0B0E0E3E2A9
:101C4000FEE00C943123288739874A875B876C87AD
:101C50007D878E87CE0108968ADE6C85811599F086
:101C6000611539F0288539854A855B857D858E85A6
:101C700090DC8091D0019091D10189133DC02E96C6
:101C8000E3E00C944D2387E09E01285F3F4FF9016C
:101C900027503109D90101900D928A95E1F761151C
:101CA00041F3A091D1018A2F90E08395877090E055
:101CB000AC012091D0012417150691F097E09A9F6E
:101CC000D0011124AE52BE4F9E012F5F3F4FF9014C
:101CD00001900D929A95E1F74093D101AFDDC9CF04
:101CE0001EDC1092D1011092D001EAE0F2E087E010
:101CF00011928A95E9F7BDCF17E0189FC001112412
:101D00008E529E4F34DE811509F4B9CFE091D00197
:101D10001E9FF0011124EE52FE4F2081318142813D
:101D2000538164817581868134DC8091D0019091EA
:101D3000D101019687708093D0019BCF80913902A9
:101D400086958695869508958091390287700895C5
:101D500090913902977081E0911101C080E008955F
:101D600080916502089590916502982B9093650289
:101D700008958095982F809165028923809365024C
:101D8000089510926502089590916402982B9093A3
:101D9000640208958095982F80916402892380932E
:101DA000640208951092640208950895FECF089584
:101DB00090913A02292F282329F080958923809336
:101DC0003A02F4CF08950895FECF089590913B0212
:101DD000292F2823281721F0982B90933B02F4CF2A
:101DE000089590913B02292F282329F0809589237B
:101DF00080933B02E9CF089580913B02811521F049
:101E000010923B0280E0E0CF0895CF93C09165022D
:101E100080916402C82B80913B02811529F0C82B68
:101E20000E94A3188111E8DF8C2FCF910895CF93E2
:101E3000DF93C0910401D0910501E7DF8883C09151
:101E40000401D091050148E050E061E372E0CE0169
:101E50000E945923892B59F088E0FE01A1E3B2E0EA
:101E600001900D928A95E1F7CE010E942918DF9129
:101E7000CF910895CF93DF93C0910201D0910301D8
:101E8000C4DF8983C0910201D091030140E250E098
:101E900061E172E0CE010E945923892B59F080E262
:101EA000FE01A1E1B2E001900D928A95E1F7CE0129
:101EB0000E943618DF91CF9108950E941118811564
:101EC00029F08091C40287FF01C0D4CFB0CF08951C
:101ED000FECF08959091C50292FF0EC0982F990FE2
:101EE000990F990F962B9093390298DB80913902C4
:101EF000869586958695ECCF91CB1092390280E03D
:101F0000E7CF909139028095892380933902282F59
:101F1000277059F4891749F09091C50292FF05C0C6
:101F200086958695869588DBE8CF08959091C502C1
:101F300092FB222720F9281749F080FB92F9909311
:101F4000C50284EC92E03FD082E0DBCF089580911F
:101F5000C502002482FF0394802DE8CF81E0E6CF04
:101F600080E0E4CF80E090E0BC019AC3A3E0B0E061
:101F7000ECEBFFE00C94322342D34DD31B82CE0115
:101F8000039660D381E090E08093CE011092CF0160
:101F900065D3198284E18A83CE01019670D30E94B1
:101FA00090042396E2E00C944E23E0CF089539C3C9
:101FB000089526C308953BC308954AC308954EC3A8
:101FC000089551C308955BC3089560C3089562C323
:101FD00008956CC30895A6E0B0E0E1EFFFE00C9433
:101FE00030230E94D21A8C01809166029091670280
:101FF0008017910779F019821A820E94D21ABC01C7
:1020000049815A8180E090E00E9441070093660276
:10201000109367022696E4E00C944C230E94DE1A8B
:1020200060936C0270936D0280936E0290936F02C6
:10203000609368027093690280936A0290936B02C6
:10204000089508950895FDCF08950895FEDFFBCF0C
:102050000C946C0508950895FEDFFACF87EB92E1AA
:10206000E7D3F0DFF3CF81E0089581E00895FBCF5F
:102070000895089508950895FCDFFCDFFCCF99DFF3
:10208000811101C092DF80E792E095DF84EC92E05D
:1020900098DF93DF95DA8091CC019091CD01A7CAAA
:1020A0000E94C91A11D3EBDFBAD70E942107D4CFFF
:1020B000A6E0B0E0EEE5F0E10C942923D6DF811133
:1020C00009C089DFADD728D60E9429072696EBE004
:1020D0000C9445230AD386EBA82E82E0B82E750116
:1020E00010E0F7010081812FE8D21F5F1E3009F454
:1020F00045C09FEFE91AF90A081799F38091700219
:1021000081FDE1D2B4DF982E10E0812FD6D2F82ED7
:10211000F50181915F01F81661F18F25D82E00E05D
:10212000EE24E3948D2D8E21F1F0CC24C3948F2DD9
:102130008E2109F4C12C911489F0602F812F0E9407
:102140003F1A81110BC009831A830E94D21ABC0165
:1021500049815A8181E09C2D0E9441074C2D602FBE
:10216000812F0E94531A0F5FEE0C0630D9F6F5014D
:10217000F2921F5F1E3049F651DFA4CF0813BECF85
:10218000A0CF0F931F93CF93DF93FDD0EC01D235F7
:1021900008F050C0D03508F0C8C0C03ED10530F5B9
:1021A000CD3CD10508F09DC0C83AD10578F4C53AB8
:1021B000D10508F093C0C130D105B1F1CE0104972B
:1021C000813A910588F1C0E0D0E02EC0CE01885A56
:1021D00091094B97C0F7C85AD0E0CC0FDD1FCF5AFA
:1021E000DE4F0990D881C02DD4641EC0D034A8F42D
:1021F000D03208F0ADC0C83ED105B0F0CE0191504C
:102200009F3108F78D2F62D1082F8C2F90E0BBD023
:10221000D02FDF71C82FD92B07C08C2F90E0B3D0FF
:10222000DF70C82FD92BD06ACE01DF91CF911F91DB
:102230000F910895C03882E5D807B8F5C03682E519
:10224000D80708F056C0C03482E5D807C8F4C032B9
:1022500082E5D80708F047C08C2F8695869520E246
:10226000829FC0011124C37021E030E002C0220F20
:10227000331FCA95E2F7E901C82BD92BDD68D4CF0B
:102280008C2F86958695877020E2829FC00111244D
:10229000C37021E030E002C0220F331FCA95E2F77D
:1022A000E901C82BD92BDC68BFCFC03C82E5D80739
:1022B00050F48C2F8F71C03AD24580F5982F84EF5F
:1022C000906AEC01B1CFCE01805C9245809708F016
:1022D0007ACFDC2FDF71C0EFD06AA6CFA497D0648D
:1022E000A3CFD065A1CF8C2F8F71D82FC1EFD06A2B
:1022F0009BCF8C2F86958695877020E2829FC001A8
:102300001124C37021E030E002C0220F331FCA95B0
:10231000E2F7E901C82BD92BDA6886CFD7D0982FFE
:1023200080E09F71EC01D0627FCF8C2F8F71CED077
:1023300053E0CC0FDD1F5A95E1F7DF70282F84FFA3
:1023400004C090E1899F90011124C22FD0696CCF05
:102350008D2F8F71BBD0082F8C2F90E014D0302F91
:102360003F71282F392B3062E9015ECF462F7E3036
:1023700028F4663018F4672F0C94AB0580E090E0E9
:102380000895F4DFFECE803E9105D1F1C8F481338B
:10239000910509F481C048F48932910509F471C0AE
:1023A0008A32910509F47FC0089589339105E1F0DF
:1023B00082389105C9F08533910509F45DC008950F
:1023C000843E9105D1F148F4823E910531F1833E7E
:1023D000910541F181EE90E00895863E9105C1F1AD
:1023E000873E9105F1F108952091C402237009F010
:1023F00064C02091C50223FF14C089E290E00895D3
:102400002091C40220FD45C03091C50230FF09C0B3
:1024100024FD24C083EE90E008952091C40222FDA3
:10242000F7CF08952091C40222FD44C03091C50227
:1024300030FD43C024FFF5CF11C02091C50221FF1C
:10244000F0CF8091C40284FD09C087EE90E008952A
:102450002091C40223FFE5CF24FFF7CF80E090E076
:1024600008952091C40223FD2BC03091C50231FF95
:10247000E1CF84EE90E008952091C40225FFD1CFF2
:10248000BCCF2091C40225FD1EC02091C50223FFB0
:10249000C8CF89E390E008952091C40226FFC1CF00
:1024A0008AE290E008952091C40226FFBACF81E32A
:1024B00090E0089582EE90E0089580EE90E0089517
:1024C00086EE90E0089585E390E008959091C4022F
:1024D00092FF10C041E0282F2471243009F040E021
:1024E00031E0282F2871283009F030E0431711F02F
:1024F0002CE0822793FF10C041E0282F2471243163
:1025000009F040E031E0282F2871283109F030E04F
:10251000431711F02CE082273091C50230FF10C024
:1025200051E0282F2171213009F050E041E0282F9F
:102530002871283009F040E0541711F029E0822773
:1025400031FF10C041E0282F2171213109F040E016
:1025500031E0282F2871283109F030E0431711F0BD
:1025600029E0822794FF02C083FD877E089580E0E2
:102570000895CF939C01205E3245C1E020323105A1
:1025800038F4FB01C581C11103C08F710E94C306DD
:102590008C2FCF9108959C01FB018581811599F0C5
:1025A0002B359CE7390769F02C359CE7390721F07A
:1025B0002A353C4721F00895CADC80E00895CEDC3E
:1025C000FCCFCEDCFACF81E008959C01FB01858130
:1025D000811599F021309CE7390761F023309CE7A1
:1025E000390739F021153C4749F40E94E20680E0A2
:1025F0000895DDDC0E94E606FACF81E00895089593
:1026000080E090E00E9473239C0181E0233E3E4FD6
:1026100009F080E0089563EE7EEF80E090E00C9496
:1026200092236FEF7FEF80E090E00C949223CF93A2
:10263000DF93EC0182E090E00E9466238883DF91C3
:10264000CF910895FC01608182E090E00C947823A2
:1026500083E090E00E94662390E00895682F83E075
:1026600090E00C947823CF93DF93EC0184E090E02A
:102670000E94732388839983DF91CF910895FC0191
:102680006081718184E090E00C9492238FE090E06F
:102690000C946E23AB01BC018FE090E00C948A2374
:1026A000AB01BC0183E190E00C948A23682F8EE09B
:1026B00090E00C94782308950895E82FF0E0EC5210
:1026C000FD4F8081089508950E940603E6ECF2E034
:1026D0008EE011928A95E9F7E4EDF2E08EE0119236
:1026E0008A95E9F713D00C942404CF9386EC92E0FA
:1026F0000E940D03482F64ED72E086EC92E007D053
:10270000C82F0E94A4048C2FCF9108950895EF92B2
:10271000FF920F931F93CF93DF93182F092FF62E5D
:10272000E72EC42F10927302D0917502D11509F4CF
:1027300069C038D740917102509172029C01241BEC
:10274000350B809371029093720284179507C9F03C
:10275000C90191118FEFE6E7F2E020E030E09191BE
:10276000911539F0DF011197891708F447C01C92C1
:102770003D2F92E0E438F90791F7309374022093EB
:102780007502C1110CC0CD2F80917402811579F1B1
:10279000C11105C007D78093710290937202109205
:1027A00074028091730290917502EF2DFE2DC12F5E
:1027B000D02F06E712E0AF01425F5F4F39E1619130
:1027C0002991621759F0D8016C91611107C03C93AF
:1027D000CF010197DC012C9381E091E00F5F1F4F47
:1027E000E417F50761F79093750280937302809167
:1027F0007302CDB7DEB7E6E00C944A23981B9C9396
:102800002D2FB7CF411509F4BFCFC4CF51CC0895B8
:1028100063D60E94F21D22DC0E940A1E41DC0E9447
:10282000131E0E94161EF2DF0E942C1E25DCF9CF1B
:1028300080939601909397010895CF93DF93EB01D6
:1028400086319C47F9F48CDA9D81911591F08A7A52
:1028500091E0811101C090E090938402811539F0DC
:1028600085E31DD52ADB80E0DF91CF91089589E2D1
:10287000F8CF80918402811519F085E327D5F2CF36
:1028800089E2FCCF81E0F0CFCF93DF93EC01FB0135
:102890008581811509F4C8C09E0130572332310566
:1028A00008F0A8C084EC92E08CDBFE01E150F04718
:1028B000E232F10520F4E652FC4D0C941C23809189
:1028C000C40281608093C4028FC08091C502886079
:1028D0008093C50289C08091C4028260F3CF809149
:1028E000C4028460EFCF8091C4028860EBCF8091F6
:1028F000C5028160EDCF8091C5028260E9CF8091F1
:10290000C4028061DFCF8091C4028062DBCF8091FE
:10291000C4028064D7CF0E948F0A8091C40280686D
:10292000D1CF8091C4028C60CDCF8091C5028360ED
:10293000CFCF8091C4028E7FC5CF8091C502877FA3
:10294000C7CF8091C4028D7FBDCF8091C4028B7FA1
:10295000B9CF8091C402877FB5CF8091C5028E7FA9
:10296000B7CF8091C5028D7FB3CF8091C4028F7E97
:10297000A9CF8091C4028F7DA5CF8091C4028F7BA7
:10298000A1CF0E948F0A8091C4028F779BCF809144
:10299000C402837F97CF8091C5028C7F99CF90919D
:1029A000C402892F8B7F92FF8460877F92FF8860AB
:1029B00089CF8091C502982F909590FB80F990FB6C
:1029C00081F986CF9091C402892F8F7B96FF806416
:1029D00079CF0E948F0A9091C402892F97FB87F9C3
:1029E000805870CF81E0F5DA84EC92E0ECDA0E9456
:1029F0008F0A80E0DF91CF91089580E0F4CF90912D
:102A0000C402892F8F7E94FF80615CCF9091C402B5
:102A1000892F8E7F90FF816055CF9091C502892FBD
:102A2000877F93FF886054CF81E0E4CF382F25EB78
:102A30003203C001112497FF04C080589109892FE7
:102A4000089580589F4FFBCF80918C0280FF0DC06E
:102A500060910B0170E0660F771F6038710588F593
:102A60006115710581F1862F089581FF07C060917E
:102A70000B0184E0689FB0011124EFCF82FF04C0F6
:102A800060910B0188E0F6CF90918B029115B9F01F
:102A900060910A0180910B01961728F098E0899FB8
:102AA000B0011124DACF899FC001112423E0880FDF
:102AB000991F2A95E1F770E00E940923CECF68E0C4
:102AC000D2CF8FE7089581E0089580918C0280FF36
:102AD0000CC06091070170E07595679575956795D5
:102AE0006115710541F1862F089581FF06C060913F
:102AF000070170E075956795F3CF6091070182FD3E
:102B00000BC090918A029115A1F06091060180910D
:102B10000701961738F0682F70E06038710500F3F0
:102B20008FE70895899FC001112470E00E94092356
:102B3000F4CF61E0D8CF81E00895E82FED5CE33178
:102B400098F5F0E0E450FC4D0C941C237DDF81955A
:102B500080938F02089578DFFBCF76DF8195809395
:102B60008E02089571DFFBCFB0DF8093900208954D
:102B7000ACDF8195FACFA9DF81958093910208950A
:102B8000A4DFFBCF815D990B21E001C0220F8A9564
:102B9000EAF780918D02822B80938D0208958091B7
:102BA0008C02816080938C02089580918C028260F7
:102BB000F9CF80918C028460F5CF40918E028D3CDC
:102BC00059F480918F0287FF0DC010928F0241153A
:102BD00059F410928B0208C08E3C81F480918F02D0
:102BE00018169CF3411581F080919002909191020A
:102BF000892B09F056C010928A0208958F3C41F447
:102C000047FFF0CF10928E0280918F028115E0CFA6
:102C1000803D19F41416B4F3E5CF90919002893DEC
:102C200029F41916FCF610929002DCCF8A3D19F4B3
:102C300097FFD8CFF8CF909191028B3D29F497FF61
:102C4000D1CF10929102CECF8C3D19F41916CCF34E
:102C5000C9CF982F915D983078F4815D990B21E070
:102C600001C0220F8A95EAF7822F809590918D02FC
:102C7000892380938D02B6CF8D3D31F480918C02F3
:102C80008E7F80938C02AECF8E3D21F480918C029A
:102C90008D7FF7CF8F3D09F0A5CF80918C028B7F80
:102CA000F0CF08957FD49C0190918E0280918F0285
:102CB000982B21F020938802309389029091900202
:102CC00080919102982B21F0209386023093870205
:102CD0008DE892E0DDC1EDE8F2E085E011928A95A1
:102CE000E9F710928B0210928A0210928C020895DA
:102CF000FC01818181110EC0828181110BC0838111
:102D0000811108C091E08481811101C090E0892F78
:102D10008170089581E0FCCFA5E0B0E0E2E9F6E142
:102D20000C942F2385E0EDE8F2E09E012F5F3F4FEA
:102D3000D90101900D928A95E1F710928E021092BE
:102D40008F0210929002109291028A819B81892BAE
:102D5000022FF32E811581F08091880290918902D3
:102D6000B2D3AC0190918B029115A1F180910C012D
:102D70008417150608F43BC08C819D81892B89F04E
:102D800080918602909187029ED3AC0190918A0235
:102D9000911509F45AC0809108018417150608F4AA
:102DA00062C0602F7F2D8DE892E0BFD2811104C0F8
:102DB0008DE892E09DDF811175DF85E0E02FFF2D2A
:102DC000ADE8B2E001900D928A95E1F72596E5E035
:102DD0000C944B23209185028AE0289F90011124B6
:102DE0002417350748F69F5F90938B0202C09F3FE0
:102DF000D1F71A81111551F027DE91E011160CF070
:102E00009FEF899F802D112480938E021B811115C5
:102E100051F01ADE91E011160CF09FEF899F802D82
:102E2000112480938F0280918E02811509F4A4CF22
:102E300010918F02111509F49FCFF8DD80938E0257
:102E4000812FF4DD80938F0297CF209109018AE0D2
:102E5000289F900111242417350708F0A2CF9F5F07
:102E600090938A0202C09F3FD1F71C81111551F047
:102E70002CDE91E011160CF09FEF899F802D11241C
:102E8000809390028D81182F811551F01EDE91E004
:102E900011160CF09FEF899F802D112480939102D1
:102EA00080919002811509F47CCF90919102192FA5
:102EB000911509F476CFBADD80939002812FB6DDAB
:102EC000809391026ECF0F931F93CF93DF93C42F04
:102ED000D22FFC0185818115C9F04093940262D301
:102EE00080939202909393028C2F805E883048F4F6
:102EF00081E0C1FD84E0C0FD880FC2FD82950E9483
:102F00007508DF91CF911F910F9108951091940250
:102F1000141333C08091920290919302D4D2883CD2
:102F2000910558F5CD2FC05E1D17C1F0812F805E31
:102F3000883048F481E011FD84E010FD880F12FD17
:102F400082950E947A08C83048F481E0D1FD84E07F
:102F5000D0FD880FD2FD82950E947508802F0E94B7
:102F60006E0881E0D1FD84E0D0FD880FD2FD82950E
:102F7000C83038F60E947A08C4CF8C2F805E883023
:102F800008F0BFCF81E0C1FD84E0C0FD880FC2FD25
:102F90008295F0CF0F93FC01CB01E851FC47E7305D
:102FA000F10588F5E15FFB4D0C941C2306E221EE50
:102FB00041EE6AE17CE787DF80E00F91089507E248
:102FC00025EE45EE6BE17CE7F6CF06E221EE40EE22
:102FD00068E17CE7F0CF07E225EE44EE69E17CE7AB
:102FE000EACF06E221EE42EE6CE17CE7E4CF07E2B5
:102FF00025EE46EE6DE17CE7DECF08E221E045EE0E
:103000006EE17CE7D8CFFB0185818111109294029B
:1030100081E0D3CF8093990290939A020895089506
:103020000895E8D1982F81E0913009F080E008956B
:10303000E0919902F0919A02309739F00190F08175
:10304000E02D309711F00995089580E00895F0CFB4
:103050000895E0919902F0919A02309731F0028040
:10306000F381E02D309709F009950895E0919902D8
:10307000F0919A02309759F024813581232B39F051
:1030800026E0DC012C930480F581E02D099508955C
:10309000E0919902F0919A02309731F00680F78121
:1030A000E02D309709F009950895A3E0B0E0EBE535
:1030B000F8E10C943223209197023091980228175E
:1030C0003907B1F08093970290939802E0919902AA
:1030D000F0919A02309761F00084F185E02D3097ED
:1030E00039F023E029838A839B83CE0101960995D9
:1030F0002396E2E00C944E23A3E0B0E0E2E8F8E18E
:103100000C943223209195023091960228173907AA
:10311000B1F08093950290939602E0919902F0911C
:103120009A02309761F00084F185E02D309739F0F4
:1031300024E029838A839B83CE01019609952396F7
:10314000E2E00C944E23CF93DF93C0910401D09121
:10315000050167DF811521F08091C40287FD11C050
:103160009E012E5F3F4F96E080E09150F901408133
:103170002F5F3F4F41118F5F9111F7CFDF91CF91BB
:10318000089520910201309103012E5F3F4F9EE18F
:10319000EBCFCF93C82F811102C080E02EC041DF5A
:1031A000811521F08091C40287FD0FC08091040138
:1031B00090910501FC013296089620812C17F9F0B8
:1031C0003196E817F907C9F7E8CF8C2F86958695D1
:1031D0008695C03F10F7E0910201F0910301E80FDE
:1031E000F11D228130E0C77081E001C0880FCA95CF
:1031F000EAF7282381E0232B81F2CF91089581E023
:10320000FCCF9C01FC01329680E09FEF4081461785
:1032100059F031969F3F19F4411101C0982F8F5FEB
:103220008630A1F79F3F09F40895290F311D97FDBE
:103230003A95F90162830895FC013296089621912E
:10324000261302C0DF011E92E817F907C1F708959F
:10325000262F269526952695603F60F4820F911DB6
:10326000FC01677021E001C0220F6A95EAF78281B4
:10327000822B82830895262F269526952695603FDA
:1032800068F4820F911DFC019DEF61FD97EF60FFD7
:10329000959562FD92958281892382830895CF93CB
:1032A000C82FBFDE6C2F811559F08091C40287FFB3
:1032B00007C08091020190910301CADFCF91089568
:1032C00080910401909105019CDFF8CFCF93C82F26
:1032D000A8DE6C2F811559F08091C40287FF07C0CA
:1032E0008091020190910301C6DFCF9108958091F2
:1032F000040190910501A0DFF8CF93DE811571F0F4
:103300008091C40287FF0AC0E0910201F09103019D
:1033100032968EE111928A95E9F70895E0910401C1
:10332000F0910501329686E0F5CFDC01FB019C911E
:103330008081981322C011968C911197811519F0F4
:10334000918189131AC012968C911297811519F0E8
:103350009281891312C014968C911497811519F0DB
:10336000948189130AC013969C91911521F081E0F4
:103370002381291303C080E001C081E0817008959A
:103380000895FECF08958F5F8093100160910D0125
:1033900070910E0180910F0190911001F2CF83E0A6
:1033A0008093100160910D0170910E0180910F01C9
:1033B00090911001E6CFE7CF089581E0809310014E
:1033C00060910D0170910E0180910F01909110019B
:1033D000D8CFF3CF089591E0811101C090E0909390
:1033E0000F0160910D0170910E0180910F0190917C
:1033F0001001C7CF80910F01089580930E01609155
:103400000D0170910E0180910F0190911001B9CFC3
:1034100080910E01089580930D0160910D017091CE
:103420000E0180910F0190911001ABCF80910D01A1
:10343000089508950895FECF08950895FACF089548
:103440000F931F93CF93DF930E94B8034ED9F5DFFC
:103450000BE912E0C0E0D0E08C2F2FD9F801819366
:103460008F0191E0811101C090E0D92BCF5FCE3068
:1034700099F78D2FDF91CF911F910F910895E82F2C
:10348000F0E0E556FD4F808190E021E030E002C0A1
:10349000220F331F6A95E2F72823392381E0232B7B
:1034A00009F480E0089541110DC0E82FF0E0E556E1
:1034B000FD4F21E001C0220F6A95EAF72095808137
:1034C000282320830895CF93DF93EC016BD08C1BCE
:1034D0009D0BDF91CF91089585B7806885BF85B733
:1034E000806885BF08951F921FB61F9211248F9385
:1034F0009F93AF93BF938091A902811113C08091D4
:10350000E2029091E302A091E402B091E5024196BB
:10351000A11DB11D8093E2029093E302A093E40207
:10352000B093E502BF91AF919F918F911F901FBE05
:103530001F9018958091EA02843031F10E94EA06CA
:103540001092A90288E190E020E40FB6F894A895C3
:10355000809360000FBE2093600083B7817F8460FA
:1035600083BF83B7816083BF7894889583B78E7F4C
:1035700083BF0FB6F894A89580916000886180930E
:103580006000109260000FBE08950E948F0A0C9494
:10359000EE0682E084BD93E095BD9AEF97BD8093DF
:1035A0006E0008952FB7F8948091E2029091E302A3
:1035B000A091E402B091E5022FBF08952FB7F894CF
:1035C0006091E2027091E3028091E4029091E50241
:1035D0002FBF089578941F921FB61F9211248F93C6
:1035E0009F93AF93BF938091E2029091E302A091E9
:1035F000E402B091E5020196A11DB11D8093E202A3
:103600009093E302A093E402B093E502BF91AF91DF
:103610009F918F911F901FBE1F901895F89481E085
:103620008093E00080E28093D800E9ECF0E0108223
:103630008FE19EE40197F1F700C000001DBA1092DF
:1036400068001CBC10BE1FBA10927A0010926E0067
:1036500010926F0010927100109272001082ECEBC9
:10366000108214B817B81AB81DB810BA108215B85D
:1036700018B81BB81EB811BA0C94003F089588E121
:103680009AE00FB6F894A895809360000FBE9093CF
:103690006000FFCFEF92FF920F931F93CF93DF93C2
:1036A000C82F8B011092BC0084EA8093BC007ADFA3
:1036B0007C018091BC0087FF25C08091B900887F84
:1036C000883029F08091B900887F803161F5C093FE
:1036D000BB0084E88093BC0065DFEC018091BC00F6
:1036E00087FF1BC02091B900287F80E090E028313F
:1036F00081F081E090E0203409F480E0919581959B
:10370000910907C0C701DFDE0817190790F68EEF91
:103710009FEFCDB7DEB7E6E0BDC7CE01D4DE081718
:103720001907E0F6F4CF8FEF9FEFF3CF1092B900B7
:103730008CE08093B80008950F931F93CF93DF938D
:10374000EB018093BB0084E88093BC002BDF8C01ED
:103750008091BC0087FF10C02091B900287F81E0D4
:1037600090E0283209F480E0919581959109DF91EC
:10377000CF911F910F910895CF3FDC0749F3C80106
:10378000A2DEC817D90720F78EEF9FEFF0CF0F9377
:103790001F93CF93DF93EC0184EC8093BC0002DF96
:1037A0008C018091BC0087FF08C08091BB0090E035
:1037B000DF91CF911F910F910895CF3FDC0789F3DF
:1037C000C80181DEC817D90760F78EEF9FEFF0CFF1
:1037D0000F931F93CF93DF93EC0184E88093BC0099
:1037E000E1DE8C018091BC0087FF08C08091BB00A6
:1037F00090E0DF91CF911F910F910895CF3FDC07AB
:1038000089F3C80160DEC817D90760F78EEF9FEF14
:10381000F0CF6F927F929F92AF92BF92CF92DF9242
:10382000EF92FF920F931F93CF93DF937B015A0187
:1038300089018160982EB6DE3C010431110578F1D2
:103840000F3F100781F1C80164E170E0CED66B0133
:10385000B601892D1FDFEC01892B41F5C12CD12C3C
:1038600081E0A81AB108CA14DB04B0F5D7FF27C05D
:1038700084E98093BC00CE011C161D0614F480E080
:1038800090E0DF91CF911F910F91FF90EF90DF902B
:10389000CF90BF90AF909F907F906F900895CC2471
:1038A000C394D12CD5CF85E0C82EFBCF0F3F100796
:1038B00079F2C30108DE0817190750F6CFCFC80107
:1038C00066DFEC0197FD04C0F701EC0DFD1D808360
:1038D0008FEFC81AD80AC7CFD7FDCACFC80178DF83
:1038E000EC0197FD05C0EA0CFB1CF7018083C0CFFB
:1038F000CEEFDFEFBDCFA0E0B0E0E0E8FCE1A6C690
:10390000B82EA62E942E852E6901E8014BDE3C01CF
:103910000431110500F10F3F100709F1C80164E1FE
:1039200070E063D6F62EE72E6F2D7E2D8B2DB2DE46
:103930008C01892BB9F0CF3FDC07B1F3C301C3DDA4
:10394000C817D90788F784E98093BC00C801CDB7B0
:10395000DEB7EEE097C6FF24F394E12CE5CF85E0D7
:10396000F82EFBCFBE018A2DE7DE8C01E92CF82C66
:10397000CE0CDF1CEC14FD0431F30115110519F711
:10398000BE01F70181917F01D7DE8C01F3CF9B014E
:10399000BA019091EA029430D9F48F708093E900D3
:1039A0009FEF8091E80085FD06C085ED8A95F1F7CF
:1039B00000009150B1F78091E80085FF09C040E018
:1039C00050E0C901BDD18091E8008E778093E80076
:1039D000089543E050E0BC0183E0D9CF45E050E0DA
:1039E000BC0182E0D4CF40E250E0BC0183E0CFCF05
:1039F000CF93DF93EC01FEDC48E050E0BE0181E0B4
:103A0000C6DF88E0FE01AAEAB2E001900D928A9535
:103A1000E1F7DF91CF9108958091E902811107C00C
:103A200016D366D38091E20084608093E20008950B
:103A30001092E9020895C1DC81E0CDCC6091E602EC
:103A400081E0611101C080E0AACC9091EA0281E09E
:103A5000943009F080E06091E602ADCC42E061EC88
:103A600081E071D242E161EC82E06DD242E261EC30
:103A700083E069D29091EA0281E0943009F080E01D
:103A80006091E60280CC8091EC02893081F148F4AB
:103A9000823009F497C0833009F458C0813041F076
:103AA00008958A3009F481C08B3009F469C0089503
:103AB0008091EB02813A09F048C08091E800877F4D
:103AC0008093E8008091EF029091F002892B59F0E9
:103AD00060E080E090E070E07FD18091E8008B773B
:103AE0008093E800089568E08AEA92E0F4CF80913C
:103AF000EB02813251F58091EF029091F0028D7FBF
:103B0000892B19F58091E800877F8093E8008091E8
:103B1000E80082FF16C02091F3008091F200922FFE
:103B2000029731F48091F100813011F0863019F460
:103B30008091F10062DC8091E8008B778093E8004F
:103B400036C28091EA028111E2CF08958091EB02A2
:103B5000813AD9F78091EF029091F002892BA9F771
:103B60008091E800877F8093E8008091E80080FFE3
:103B7000FCCF40DC8093F1008091E8008E77DECFAF
:103B80008091EB02813209F78091EF029091F0026F
:103B9000892BD9F68091E800877F8093E80007D2CF
:103BA0008091ED0218DC0C948F0A8091EB02813237
:103BB00061F68091E800877F8093E800F8D18091DA
:103BC000EE0229CC8091EB02813A09F0BECF8091C0
:103BD000E800877F8093E8008091E80080FFFCCFB9
:103BE00025DCC8CF84B7877F84BF0FB6F894A8952B
:103BF00080916000886180936000109260000FBE29
:103C000080E890E00FB6F894809361009093610093
:103C10000FBEDFCB1CD26CD2E2EEF0E0808184607C
:103C200080837894C9C481E191E0F4C98091EA026B
:103C3000853029F48091EA02853011F0A6CC0895F0
:103C400079DCFEDB8115B1F38091E802811591F3F7
:103C500061D00E948F0AEECF08959A014091F1023F
:103C60005091F20200C0492F50E043305105D1F08D
:103C700078F44130510509F448C04230510571F4DF
:103C800084E590E04AE354E0F901408351830895CC
:103C900041325105E9F04232510539F180E090E0BE
:103CA00040E0F2CF482F50E0813061F042305105C2
:103CB00061F0E6E3F4E04115510581F7849190E06D
:103CC000AF01E2CFECE0F4E0F9CFE4EFF3E0F6CFC0
:103CD0006330710518F7660F771FFB01E057FE4F41
:103CE0004081518189E090E0CFCF63307105B0F61B
:103CF000FB01EE0FFF1FE657FE4F408151816957D0
:103D00007E4FFB01808190E0BFCF82E190E04EE8E2
:103D100054E0BACF80E189BD82E189BD09B400FEDB
:103D2000FDCF8091D8008F7D8093D8008091E000F6
:103D300082608093E0008091E00081FDFCCF0895D7
:103D4000AF92BF92CF92DF92EF92FF921F93CF93E9
:103D5000DF937C01EB016A0149D1182F811122C048
:103D6000C114D10439F0F60180819181C81BD90BAF
:103D7000E80EF91EA12CB12C2097A1F08091E8004B
:103D800085FD20C08091E8008E778093E800C11403
:103D9000D10499F0F601808191818A0D9B1D808369
:103DA000918315E0812FDF91CF911F91FF90EF90CC
:103DB000DF90CF90BF90AF90089518D18115F1F2A8
:103DC000182FF0CFF70181917F018093F1002197A7
:103DD0008FEFA81AB80AD0CFFC018091F102909120
:103DE000F2028617970720F06115710561F0CB018B
:103DF00040E0009771F441110CC08091E80082FF0F
:103E000036C080E008958091E8008E778093E800C6
:103E1000EECF2091EA022115B1F12530B1F12091C8
:103E2000E80023FD2EC02091E80022FDE6CF20917E
:103E3000E80020FFDECF4091F3002091F200342F04
:103E4000009719F02830310558F041E0283031054D
:103E500009F040E02091E8002E772093E800C9CFD8
:103E600041914093F10001972F5F3F4FE9CF80913F
:103E7000EA02811541F0853041F08091E80083FF2E
:103E8000BCCF81E0089582E0089583E00895FC01AD
:103E90008091F1029091F2028617970720F0611548
:103EA000710561F0CB0140E0009771F441110CC045
:103EB0008091E80082FF37C080E008958091E8009B
:103EC0008E778093E800EECF2091EA022115B9F1B8
:103ED0002530B9F12091E80023FD2FC02091E800A2
:103EE00022FDE6CF2091E80020FFDECF4091F300D5
:103EF0002091F200342F009719F02830310558F046
:103F000041E02830310509F040E02091E8002E77AB
:103F10002093E800C9CF44914093F1003196019776
:103F20002F5F3F4FE8CF8091EA02811541F0853045
:103F300041F08091E80083FFBBCF81E0089582E0EB
:103F4000089583E00895982F973028F08F7080931C
:103F5000E90081E008959093E900242F762F50E046
:103F6000981731F07091EC002091ED005091F00025
:103F700021FD02C09F5FE8CF3091EB003E7F309380
:103F8000EB003091ED003D7F3093ED003091EB0080
:103F900031603093EB007093EC002093ED00509370
:103FA000F0002091EE0027FDE5CF80E0089580919C
:103FB000EB0287FF13C08091E80082FF06C080916A
:103FC000E8008B778093E80008958091EA028111E0
:103FD000F2CF08958091EA028115D9F38091E8002B
:103FE00080FFF8CF8091E8008E77ECCF2091E4003D
:103FF0003091E50095E6A9012091EC00822F8170B7
:1040000020FF06C08091E80080FF06C080E0089590
:104010002091E80022FD1AC08091EA02811589F002
:10402000853089F08091EB0085FD0FC02091E40080
:104030003091E50042175307F9F29150E1F684E020
:10404000089582E0089583E0089581E008955FD0A7
:1040500066D0E0EEF0E0808181608083E8ED8081D1
:104060008F77808319BCA7EDB0E08C918E7F8C9305
:1040700080818F7E80831092E9020895CF93DF9331
:1040800046D04DD0C8EDD0E088818F778883888175
:104090008068888388818F7D888319BC1092EA02AA
:1040A0001092E6021092E8021092E702E0EEF0E0D1
:1040B00080818B7F808388818160888342E060E09B
:1040C00080E041DFE1EEF0E080818E7F8083E2EEF0
:1040D000808181608083808188608083E0EE808140
:1040E0008E7F8083888180618883DF91CF9108955E
:1040F000E8EDF0E080818F7E8083E7ED8081816054
:10410000808384E082BF81E08093E902B7CFE8ED4D
:10411000F0E080818E7F80831092E20008951092FB
:10412000DA001092E10008951F920F920FB60F92DD
:1041300011242F933F934F935F936F937F938F93AC
:104140009F93AF93BF93EF93FF938091E10082FF22
:104150000AC08091E20082FF06C08091E1008B7F5F
:104160008093E10028D28091DA0080FF18C080910E
:10417000D80080FF14C08091DA008E7F8093DA002F
:104180008091D90080FF8FC080E189BD82E189BD27
:1041900009B400FEFDCF81E08093EA023DDC80910E
:1041A000E10080FF18C08091E20080FF14C0809180
:1041B000E2008E7F8093E2008091E2008061809334
:1041C000E2008091D80080628093D80019BC85E01D
:1041D0008093EA0233DC8091E10084FF28C0809163
:1041E000E20084FF24C080E189BD82E189BD09B479
:1041F00000FEFDCF8091D8008F7D8093D800809104
:10420000E1008F7E8093E1008091E2008F7E8093B9
:10421000E2008091E20081608093E2008091E602FA
:10422000811509F445C084E08093EA020EDC809198
:10423000E10083FF27C08091E20083FF23C08091CB
:10424000E100877F8093E10082E08093EA02109290
:10425000E6028091E1008E7F8093E1008091E20090
:104260008E7F8093E2008091E20080618093E20083
:1042700042E060E080E067DE8091F000886080933B
:10428000F000D9DBFF91EF91BF91AF919F918F919A
:104290007F916F915F914F913F912F910F900FBE42
:1042A0000F901F90189519BC1092EA02C1DB77CFCE
:1042B0008091E30087FF02C083E0B6CF81E0B4CFF6
:1042C0001F920F920FB60F9211241F932F933F93BB
:1042D0004F935F936F937F938F939F93AF93BF930E
:1042E000CF93DF93EF93FF93E9EEF0E0808110919D
:1042F000EC008F7010FB112717F9182B1082C0EFFC
:10430000D0E08881877F888378941CD0E9EEF0E044
:1043100010828881886088831F701083FF91EF91DD
:10432000DF91CF91BF91AF919F918F917F916F91CD
:104330005F914F913F912F911F910F900FBE0F9062
:104340001F901895AAE2B0E0E7EAF1E28AC18BEE8D
:1043500092E0FC0101962091F100208322E0833F4E
:104360009207B9F790DB8091E80083FF37C0809116
:10437000EB029091EC029A3088F5E92FF0E0EA5ECA
:10438000FB4D5AC1803889F0823841F58091EF02A7
:104390008F70873018F58093E9008091EB0085FBE2
:1043A000882780F91092E90006C08091E802880F02
:1043B0009091E702892B9091E800977F9093E80015
:1043C0008093F1001092F1008091E8008E7722C076
:1043D000811115C08091ED02813001F18091E800DA
:1043E00083FF0AC08091E800877F8093E800809176
:1043F000EB0080628093EB00AA96E3E04EC182302E
:1044000069F78091ED02811579F01092E9008091B1
:10441000E800877F8093E800CADDE0CF933009F0A1
:1044200080E08093E802F1CF8091EF028F70282F17
:104430002150263098F68093E9002091EB0020FF70
:10444000E4CF933031F48091EB0080628093EB00F5
:10445000DCCF9091EB0090619093EB0021E001C0E4
:10446000220F8A95EAF72093EA001092EA008091E1
:10447000EB008860EBCF8111B1CF8091ED028F7797
:10448000182F8091E3008078812B8093E300809146
:10449000E800877F8093E8008ADD8091E80080FF54
:1044A000FCCF8091E30080688093E30083E01111EA
:1044B00001C082E08093EA0291CF8058823008F0F8
:1044C0008DCF8091ED029091EE028C3D23E092071A
:1044D00089F583E08A838AE289834FB7F894DE0105
:1044E000139620E03EE051E2E32FF0E050935700B6
:1044F000849120FF03C082958F703F5F8F708A3058
:10450000B8F0895C8D931D922F5F243169F74FBFFE
:104510008091E800877F8093E8006AE270E0CE0136
:1045200001965ADC8091E8008B778093E80056CFA3
:10453000805DE8CF6091EF027091F0029E012F5FE5
:104540003F4FA9018ADBBC01892B09F447CF909129
:10455000E800977F9093E80089819A8198DCE2CF08
:10456000803809F03BCF8091E800877F8093E80096
:104570008091E6028093F10027CF81112FCF909197
:10458000ED02923008F02ACF8091E800877F809377
:10459000E8009093E6020BDD8091E602811529F098
:1045A00084E08093EA025ADA19CF8091E30087FD14
:1045B000F7CF81E0F6CF0895CF938091EA0281157D
:1045C00091F08091E900C091EC008F70C0FBCC2786
:1045D000C7F9C82B1092E9008091E80083FDB2DE94
:1045E000CF70C093E900CF910895AA1BBB1B51E186
:1045F00007C0AA1FBB1FA617B70710F0A61BB70B53
:10460000881F991F5A95A9F780959095BC01CD01F7
:10461000089597FB072E16F4009406D077FD08D076
:10462000E4DF07FC05D03EF4909581959F4F0895F7
:10463000709561957F4F0895EE0FFF1F0590F491DF
:10464000E02D09942F923F924F925F926F927F924A
:104650008F929F92AF92BF92CF92DF92EF92FF9292
:104660000F931F93CF93DF93CDB7DEB7CA1BDB0B3E
:104670000FB6F894DEBF0FBECDBF09942A883988E3
:1046800048885F846E847D848C849B84AA84B984EA
:10469000C884DF80EE80FD800C811B81AA81B981F6
:1046A000CE0FD11D0FB6F894DEBF0FBECDBFED010A
:1046B0000895FB01DC0104C08D910190801921F463
:1046C00041505040C8F7881B990B0895F999FECFC7
:1046D00092BD81BDF89A992780B50895A6E1B0E012
:1046E00044E050E025C0A8E1B0E042E050E020C046
:1046F000262FF999FECF92BD81BDF89A019700B49B
:10470000021639F01FBA20BD0FB6F894FA9AF99A3A
:104710000FBE08950396272FECDFEADF252FE9DF90
:10472000242FE7CF0196272FE4DFE2CFDC01CB0176
:10473000FC01F999FECF06C0F2BDE1BDF89A3196B1
:1047400000B40D9241505040B8F70895F894FFCF4F
:10475000B304BA04BF04C404C904CE04D304D80407
:10476000DD04E204E704EC04F104F604FC040205B1
:1047700008050E0514051A05200526052C05320529
:1047800038053E0544054A0550055C0565057F056D
:1047900085058805840587058B058A05BA08BA084A
:1047A000F108F10847096309E208E2086709D90935
:1047B000E609E60999140615A1146B146F14A514E3
:1047C0007314A914B5147F14FF148314B914871437
:1047D000BD14E2148B14C114E9149114C714CF143E
:1047E0007714AD147B14B1149514CB14D914F214AE
:1047F000FD1465149D140D15A615AB15AD15B21558
:10480000C215C215C215C215C215C215C215C215F0
:10481000B415B815BB15C015CF15D515D915E517A5
:10482000EB17D617DF17F117F717FD17C221E8218D
:10483000EE21E821EE213B225D22EE21B022BD22B5
:1048400020003C025C023C0714283C0714000001D5
:1048500000081AF81CF31CEE1CE91CE200E900EA4F
:1048600000B500B600B700CD008301CC008A0192EC
:104870000194012102230224022502260227022A92
:1048800002B300B4006F0070009F01CB019F02A033
:1048900002E200E900EA00B500B600B700CD0083EF
:1048A00001CC008A019201940121022302240225F5
:1048B00002260227022A02B300B4006F0070009F94
:1048C00001CB019F02A00244476D54050D05A004D1
:0648D0004C0465047E04A7
:00000001FF
